:040000008A11112828
:10000800FE00030EF8000408F9000A08FA0083123B
:1000180003137F08FB008A11232D8A15202AFF303D
:1000280083120313BD00FF30BE00EE010314EE0D72
:100038000330A0000030A1006D08013EA20000308E
:1000480003180130A3008A11A5278A11831203130C
:100058002008013EAE002E08BF00C9010314C90DD7
:10006800E729003083160313AF000030AE000030DC
:10007800AD000030AC0083120313C1015E294908AA
:10008800AE00AF012E08A0002F08A1006D08FF3EAA
:10009800A200FF3003180030A3008A1516258A1124
:1000A800831203132008FF3EBB0021080318013EFA
:1000B800FF3EBC00C2014B294208AE00AF012E082A
:1000C800A0002F08A1004908B000B1013008A20023
:1000D8003108A3008A1562228A118312031341088A
:1000E8002007C7000030031801302107C80049085D
:1000F8004707C40048080318480AC5004708AE0067
:100108002E07203E840083170008AF00840A0008E9
:10011800B0004408B1003107203E84000008B20056
:10012800840A0008B30030083302031D9D282F08F5
:1001380032020318A028A128F2284708AE002E078B
:10014800203E84000008AF00840A0008B00044087C
:10015800B1003107203E84000008B200840A00087C
:10016800B300B209B309B20A0319B30A2F08320758
:10017800B40030080318300A3307B5003408B60055
:100188003508B700B801B901360883160313AC0760
:1001980083120313370803110318013E0319D728E4
:1001A80083160313AD0783120313380803110318CA
:1001B800013E0319E22883160313AE0783120313C3
:1001C800390803110318013E0319ED288316031398
:1001D800AF078312031383160313442983124408B9
:1001E800AE002E07203E84000008AF00840A0008F5
:1001F800B0004708B1003107203E84000008B20073
:10020800840A0008B300B209B309B20A0319B30A91
:100218002F083207B40030080318300A3307B50036
:100228003408B6003508B700B801B9013608831696
:100238000313AC0783120313370803110318013E95
:100248000319292983160313AD07831203133808EA
:1002580003110318013E0319342983160313AE074B
:1002680083120313390803110318013E03193F29A8
:1002780083160313AF07831203138316031344294A
:10028800013083120313AE002E08C2074B2942081F
:10029800AE00AF013C082F02031D54293B082E0273
:1002A800031C57295829602859290130AE002E0807
:1002B800C1075E2949084102031C632964294328B0
:1002C80065294908AE00AF01B001B1013108A300AA
:1002D8003008A2002F08A1002E08A00083160313DF
:1002E8002F0883120313A700831603132E08831203
:1002F8000313A600831603132D0883120313A50006
:10030800831603132C0883120313A4008A15FC23F5
:100318008A1183120313230883160313AF00831271
:100328000313220883160313AE0083120313210854
:1003380083160313AD0083120313200883160313D7
:10034800AC00831203133D08AE003E08AF00B001B5
:10035800B1013108831603132F02031DC929831223
:1003680003133008831603132E02031DC9298312B1
:1003780003132F08831603132D02031DC9298312A3
:1003880003132E08831603132C020318CC29CD2936
:10039800E229831203134908AE002E08EE008316E3
:1003A80003132D0883120313BE01BE07831603131C
:1003B8002C0883120313BD01BD07E2290130831203
:1003C800AE002E08C9073F084902031CEC29ED2995
:1003D8003528EE296E08AE002E08A0006D088A1593
:1003E800BC228A1183120313AF002F08C000C60174
:1003F800A52A003083160313AF000030AE0000308A
:10040800AD000030AC0083120313C301642A6E08E8
:10041800AE00AF012E08A0002F08A1004308B000CD
:10042800B1013008A2003108A3008A1562228A119E
:10043800831203132008B2002108B30046083207CC
:10044800B4003407203E840083170008B500840AEE
:100458000008B6003508B7003608B800B901BA0177
:10046800370883160313AC078312031338080311E4
:100478000318013E0319432A83160313AD07831299
:100488000313390803110318013E03194E2A831672
:100498000313AE07831203133A0803110318013E2E
:1004A8000319592A83160313AF07831203138316FC
:1004B8000313013083120313AE002E08C307642A06
:1004C80040084302031C692A6A2A0B2A6B2A40083F
:1004D800AE00AF01B001B1013108A3003008A2009D
:1004E8002F08A1002E08A000831603132F088312DB
:1004F8000313A700831603132E0883120313A60001
:10050800831603132D0883120313A5008316031300
:100518002C0883120313A4008A15A6248A118312B7
:1005280003134608B2003207203E840020088317D0
:100538008000840A210880000130AE002E08C6071A
:10054800A52A6E084602031CAA2AAB2AFD29AC2A52
:1005580008008312031385128316031385128B1365
:100568008A1599218A118A15AA218A118A159E212C
:100578008A118A15D1218A118A15EE228A118A15C3
:10058800E7218A118B17023083120313D70057080B
:10059800A0000230D8005808A10014308A150122A2
:1005A8008A118A158E228A11003083120313C9001A
:1005B8000030C8000130C700C230C6008A152923A0
:1005C8008A11E62A8A15AB268A11013A031DED2AFB
:1005D800EE2A2D2B143083120313D7005708A000DE
:1005E8001430D8005808A1000E308A1501228A114B
:1005F8008A158E228A11003083120313C900003035
:10060800C8000030C7001E30C6008A1529238A1189
:100618008A158E228A11003083120313C900003014
:10062800C8000030C7001E30C6008A1529238A1169
:100638008A158E228A11003083120313C9000030F4
:10064800C8000730C700D030C6008A1529238A1190
:10065800E62A8A1113208A11831203136E08D70021
:100668005707203ED8005808EF0083160313B2013D
:10067800B30183120313DF01E001E2016F2B62086B
:10068800D7005707203E840083170008D800840A43
:100698000008D9006208DA005A076F07DB005B0818
:1006A800840058088000840A590880006208D7002E
:1006B8005707203E84000008D800840A0008D900A3
:1006C8005808DF070318E00A5908E0070130D70087
:1006D8005708E2076F2B6E086202031C742B752BF8
:1006E800432B762B8A1100278A11FC3083120313BF
:1006F800D7005708EB05831603132B08831203133F
:10070800B500831603132A0883120313B400831653
:100718000313290883120313B3008316031328084D
:1007280083120313B2008A158C258A1183120313CE
:100738003508C9003408C8003308C7003208C600A5
:100748008A1529238A1183120313E3016308D7004A
:1007580057076F07D80058088400831700088316C6
:100768000313B000840A0008B1008A15BB218A115E
:1007780083120313230883160313AB008312031396
:10078800220883160313AA00831203132108831671
:100798000313A90083120313200883160313A80068
:1007A8008312031385128A158E228A11831203136A
:1007B8008516F22C83160313280983120313D70016
:1007C80083160313290983120313D800831603130E
:1007D8002A0983120313D900831603132B098312E2
:1007E8000313DA00D70A0319D80A0319D90A031917
:1007F800DA0A8A15BB218A11831203132008D70746
:1008080021080318210F092C0A2CD80722080318DD
:10081800220F0F2C102CD90723080318230ADA07F4
:1008280083160313300883120313DB0083160313A4
:10083800310883120313DC00DD01DE015A085E0271
:10084800031D302C59085D02031D302C58085C022A
:10085800031D302C57085B020318332C342C762CDC
:100868008A15BB218A1183120313230883160313E5
:10087800AB0083120313220883160313AA00831202
:100888000313210883160313A900831203132008F6
:1008980083160313A800013083120313D7005708E7
:1008A800E3076E086302031C5A2C5B2C5D2CE301E2
:1008B8005D2C6308D70057076F07D80058088400D5
:1008C8008317000883160313B000840A0008B100D8
:1008D8008312031385128A158E228A118312031339
:1008E8008516762C6B08033903197B2C7C2CF22C8B
:1008F8006B1C7F2C802C902C6E08D700D8015708D1
:1009080083160313B2070318B30A83120313580894
:1009180083160313B307902C8312EB1C942C952C8D
:10092800A52C6E08D700D801570883160313B20206
:1009380083120313580883160313031CB303B3026B
:10094800A52CFC308312D7005708EB05D32C61087F
:10095800013A031DB02CB12CC12C6E08D700D80168
:10096800570883160313B202831203135808831619
:100978000313031CB303B302D32C83126E08D700EE
:10098800D801570883160313B2070318B30A831252
:100998000313580883160313B307D32CD32C8A11D7
:1009A80000278A1183120313D7005708E100E108D2
:1009B800031DDF2CE02CAB2CE12C6308D700570774
:1009C8006F07D8005808840083170008831603139C
:1009D800B000840A0008B100F22CF22C8A153F22DC
:1009E8008A1100308312031321023D3003192002BB
:1009F800031CFF2C002DDE2B012D0030C900003018
:100A0800C8000030C700C830C6008A1529238A11DB
:100A18008A158E228A11003083120313C900003010
:100A2800C8000030C7001E30C6008A1529238A1165
:100A38008A158E228A11E62AE62A8A1111288B1E27
:100A4800262D272DF42E0B1D2A2D2B2DF42E0130AB
:100A580083160313B50255308312031381008316DE
:100A68000313B508031D392D3A2D8A2E0A30F000DC
:100A78007008B500013083120313E407003003182F
:100A88000130E507003003180130E607003003188D
:100A98000130E70703306405F00000306505F10018
:100AA80000306605F20000306705F3007308720431
:100AB80071047004031D612D622D8A2E0310FD0D33
:100AC8000310FC0D061F692D6A2D6B2D7D14861FE2
:100AD8006E2D6F2D712D7C14712DFD08031D752D44
:100AE800762DEF2D6B1D792D7A2D962D6B14FB30FD
:100AF800F0007008EB05670883160313A70083123C
:100B08000313660883160313A600831203136508EC
:100B180083160313A50083120313640883160313B3
:100B2800A400EF2D83126408F0006508F100660840
:100B3800F2006708F300831603132409F40025095B
:100B4800F5002609F6002709F700F40A0319F50A43
:100B58000319F60A0319F70A7408F0077508031849
:100B6800750FB72DB82DF10776080318760FBD2D30
:100B7800BE2DF20777080318770AF30700307302CF
:100B8800031DD02D00307202031DD02D00307102DC
:100B9800031DD02D65307002031CD32DD42DEF2DED
:100BA800831203136B14670883160313A7008312B9
:100BB8000313660883160313A6008312031365083C
:100BC80083160313A5008312031364088316031303
:100BD800A400EF2DEF2D7D08FF3A031DF42DF52D10
:100BE800FC2D83126B19F92DFA2DFC2D6B15FC2D9C
:100BF800FC08031D002E012E7B2E8312EB1D052EF3
:100C0800062E222EEB14F730F0007008EB0567086B
:100C180083160313A30083120313660883160313B2
:100C2800A20083120313650883160313A10083121D
:100C38000313640883160313A0007B2E8312640831
:100C4800F0006508F1006608F2006708F3008316F3
:100C580003132009F4002109F5002209F6002309ED
:100C6800F700F40A0319F50A0319F60A0319F70A33
:100C78007408F00775080318750F432E442EF10702
:100C880076080318760F492E4A2EF20777080318BC
:100C9800770AF30700307302031D5C2E00307202DE
:100CA800031D5C2E00307102031D5C2E653070023E
:100CB800031C5F2E602E7B2E83120313EB14670830
:100CC80083160313A3008312031366088316031302
:100CD800A20083120313650883160313A10083126D
:100CE8000313640883160313A0007B2E7B2E7C0855
:100CF800FF3A031D802E812E8A2E8312EB19852E32
:100D0800862E8A2EEB158A2E8A2E8A2E013083167D
:100D18000313B402B408031D922E932EF22E8312ED
:100D280003136C1D982E992ECB2E83160313B40132
:100D38000314B40D0130F000700883120313EC079C
:100D48006C080339033A031DAA2EAB2EB02EFC30D3
:100D5800F0007008EC05B02E6C080339683E84007A
:100D6800831300088700FB30F0007008EC050130A1
:100D7800F0006C080339013EC32E0310F00DFF3E4E
:100D8800031DC12E7008F10071088504F22E013090
:100D9800F0006C080339013ED32E0310F00DFF3E1E
:100DA800031DD12E7008FF3AF10071088505EC1D6E
:100DB800DE2EDF2EE62E0330F000700883160313B4
:100DC800B400ED2E2830F000700883160313B40029
:100DD800ED2E831203136C15F22EF22E0B11F42E46
:100DE8007B088312FF007A088A0079088400780E4D
:100DF8008300FE0E7E0E090083120313B301B401B3
:100E0800B501832F3508AD002D07203E84008317D8
:100E18000008A000840A0008A1006030A200EA309F
:100E2800A3008A11A5278A11831603133208831297
:100E380003132007A0008316031333080318330A8B
:100E4800831203132107A1006030A200EA30A30037
:100E58008A11A5278A11831203133508AE002E07BD
:100E68006F07AF002F088400200883178000840ACA
:100E7800210880003508AD002D076F07AE002E0849
:100E880084000008AF00840A0008B000C0302F05B5
:100E9800B100FF303005B20032083104031D552F70
:100EA800562F592F0130A42FA42F3508AD002D0738
:100EB8006F07AE002E0884000008AF00840A0008FF
:100EC800B000B01F682F692F6C2F0230A42FA42FF9
:100ED8003508AD002D076F07AE002E088400000806
:100EE800AF00840A0008B0002F08B3070318B40A3B
:100EF8003008B4070130AD002D08B507832F6E0800
:100F08003502031C882F892F062F8A2F3408A10148
:100F1800A1073308A001A0076030A200EA30A300AF
:100F28008A11A5278A11831203132108A901A90789
:100F38002008A801A8078A1507268A110030A42FBF
:100F4800080083120313A501A60121082004031930
:100F5800AE2FAF2FED2FA7010314A70DBF2F013020
:100F68000310A00DA10DFF3E031DB42F0130A400F6
:100F78002408A707BF2FA11FC22FC32FB32FC52F28
:100F8800C52F01300310A50DA60DFF3E031DC62F6A
:100F980021082302031DD22F20082202031CD52F6B
:100FA800D62FDE2F2008A2022108031CA303A302C8
:100FB8002514DE2F01300310A10CA00CFF3E031DE9
:100FC800DF2F0130A702031DEA2FEB2FC52FED2FCE
:100FD800ED2F2608A101A1072508A001A007F42FDD
:100FE800080064008001840A04060319003404061A
:040FF800F62F0A3492
:1010000008308A000408840A82070034A034F934C6
:1010100064347034393432342234F8342034303487
:10102000283423346734613426342E34A7346B34A7
:1010300063342C346F343234273431347734FF3412
:10133200831603130F16970108008316031306176B
:1013420086178113950183120317950115179517B7
:101352000800831603130616831203179E019F01CA
:101362001F155030831603139F00A93083120313F5
:101372009F0008008B13831203136708A7006608F7
:10138200A6006508A5006408A4008B172708A3001F
:101392002608A2002508A1002408A000D0290800E0
:1013A2007C3083160313920087160C3083120313CA
:1013B200970083160313120883120313A00003106D
:1013C200200C95008C100530920008008316031340
:1013D200811555308312031381008B160B1183166E
:1013E2000313B501003083120313E7000030E60057
:1013F2000030E5000030E400831603138112080078
:1014020083120313A3002308013E84008A150020DF
:101412008A15A2002208E8002008013E84008A15ED
:1014220000208A15A2002208E9002108013E84005A
:101432008A1500208A15A2002208EA000800FC0191
:10144200FD0183136430840070308A11F5278A15F8
:10145200A0308400B4308A11F5278A158317203012
:10146200840068308A11F5278A15831603138A11BE
:10147200FD278A15B50083018A11AD2A0330831234
:101482000313A200A20B432A831203139F14492AB7
:101492009F184C2A4D2A492A4E2A1E08A200A3014F
:1014A2002208A300A201831603131E08831203134A
:1014B2002207A0000030031801302307A100612A8F
:1014C200080083120313A401A501672A201C6A2ABB
:1014D2006B2A712A2208A4070318A50A2308A50764
:1014E20001300310A20DA30DFF3E031D722A01302D
:1014F2000310A10CA00CFF3E031D792A2108200431
:10150200031D842A852A672A862A2508A101A107A4
:101512002408A001A0078D2A08000C3083120313AF
:10152200970083160313871283120313EC150030FE
:10153200C9000030C8000030C7001930C6008A1543
:1015420029238A1583120313970187128316031323
:101552008716F73083120313D2005208EC050030CD
:10156200C9000030C8000030C7000530C6008A1527
:1015720029238A15080083120313A200A40120085C
:10158200031DC42AEB2AA3010314A30DCF2A0310BF
:10159200A00D0130A1002108A307CF2AA01FD22A43
:1015A200D32AC82AD52AD52A0310A40D200822023C
:1015B200031CDC2ADD2AE12A2008A2022414E12AE3
:1015C2000310A00C0130A302031DE82AE92AD52A40
:1015D200EB2AEB2A2408ED2A0800F83083120313C1
:1015E200A0002008831603138505F8308312031325
:1015F200A0002008850520308316031387001A30C7
:1016020084008A1500208A15831203138700EC01D7
:1016120083160313B4010314B40D1A3084008A151F
:1016220000208A1583120313A0002008E8001A3054
:1016320084008A1500208A15A0002008E9001A30CB
:1016420084008A1500208A15A0002008EA000800FC
:101652008A15BB218A158312031320084607CA0084
:101662000030031801302107CC010318CC0A4707C8
:10167200CB000318CC0A22084C07CD010318CD0A6F
:101682004807CC000318CD0A23084D074907CD00AF
:101692004D08D1004C08D0004B08CF004A08CE00BC
:1016A200532B532B8A15BB218A158312031323084C
:1016B2005102031D662B22085002031D662B2108CE
:1016C2004F02031D662B20084E020318692B6A2B5A
:1016D200532B6B2B080083120313210820040319D8
:1016E200732B742BAA2BA5010314A50D842B013097
:1016F2000310A00DA10DFF3E031D792B0130A400A4
:101702002408A507842BA11F872B882B782B8A2BD3
:101712008A2B21082302031D902B20082202031C7E
:10172200932B942B9B2B2008A2022108031CA303BA
:10173200A3029B2B01300310A10CA00CFF3E031D42
:101742009C2B0130A502031DA72BA82B8A2BAA2BA9
:10175200AA2B2308A101A1072208A001A007B12BEF
:101762000800003083120313AE000030AD000030D9
:10177200AC000030AB00AF01EB2B2F08A400240714
:10178200203E840083170008A500840A0008A600F2
:101792002508A7002608A800A901AA012708AB0767
:1017A200280803110318013E0319D82BAC07290896
:1017B20003110318013E0319DF2BAD072A08031199
:1017C2000318013E0319E62BAE070130A4002408DA
:1017D200AF07EB2B6E082F02031CF02BF12BBE2B55
:1017E200F22B2E08A3002D08A2002C08A1002B0822
:1017F200A000FB2B0800003083120313AC00003062
:10180200AB000030AA000030A900072C201C0A2CD3
:101812000B2C232C2408A907250803110318013EC9
:101822000319142CAA07260803110318013E0319F1
:101832001B2CAB07270803110318013E0319222CA6
:10184200AC07232C0130A8000310A40DA50DA60D92
:10185200A70DA80B252C01300310A30CA20CA10C80
:10186200A00CFF3E031D2D2C23082204210420047A
:10187200031D3C2C3D2C072C3E2C2C08A3002B08CE
:10188200A2002A08A1002908A000472C0800831200
:1018920003132B082A04290428040319512C522C5F
:1018A2009C2CB1010314B10D642C0130B000031063
:1018B200A80DA90DAA0DAB0DB00B582C0130B0002C
:1018C2003008B107642CAB1F672C682C562C6A2C8D
:1018D2006A2C2B082F02031D782C2A082E02031DC6
:1018E200782C29082D02031D782C28082C02031CB1
:1018F2007B2C7C2C8B2C2808AC022908031C290F7A
:10190200AD022A08031C2A0FAE022B08031C2B0F60
:10191200AF028B2C01300310AB0CAA0CA90CA80C43
:10192200FF3E031D8C2C0130B102031D992C9A2C11
:101932006A2C9C2C9C2C2F08AB002E08AA002D0888
:10194200A9002C08A800A52C08000030831203135C
:10195200AC000030AB000030AA000030A900230820
:101962002204210420040319B72CB82C0C2DAD013C
:101972000314AD0DCA2C0130A8000310A00DA10D57
:10198200A20DA30DA80BBE2C0130A8002808AD079C
:10199200CA2CA31FCD2CCE2CBC2CD02CD02C013089
:1019A200A8000310A90DAA0DAB0DAC0DA80BD22CEB
:1019B20023082702031DE72C22082602031DE72C19
:1019C20021082502031DE72C20082402031CEA2C0F
:1019D200EB2CFB2C2008A4022108031C210FA502DA
:1019E2002208031C220FA6022308031C230FA702AE
:1019F2002914FB2C01300310A30CA20CA10CA00C87
:101A0200FF3E031DFC2C0130AD02031D092D0A2DE2
:101A1200D02C0C2D0C2D2C08A3002B08A2002A0878
:101A2200A1002908A000152D080083120313A601A6
:101A3200A11F1C2D1D2D262DA009A109A00A0319E5
:101A4200A10AA6010314A60D262DA31F292D2A2DB6
:101A5200342DA209A309A20A0319A30A0130A40082
:101A62002408A606342DA701A80121082004031981
:101A72003B2D3C2D7A2DA5010314A50D4C2D0130D3
:101A82000310A00DA10DFF3E031D412D0130A40046
:101A92002408A5074C2DA11F4F2D502D402D522D4E
:101AA200522D01300310A70DA80DFF3E031D532D2B
:101AB20021082302031D5F2D20082202031C622D30
:101AC200632D6B2D2008A2022108031CA303A3028D
:101AD20027146B2D01300310A10CA00CFF3E031D37
:101AE2006C2D0130A502031D772D782D522D7A2DF4
:101AF2007A2D2608031D7E2D842DA709A809A70A81
:101B02000319A80A842D2808A101A1072708A0010A
:101B1200A0078B2D08008A15B2238A15831203139E
:101B22002308C5002208C4002108C3002008C200FF
:101B32004208B6004308B7004408B8004508B90097
:101B42004508AB004408AA004308A9004208A800BF
:101B52003209BA003309BB003409BC003509BD00A3
:101B6200BA0A0319BB0A0319BC0A0319BD0A8A156A
:101B7200BB218A15831203132008BA072108031810
:101B8200210FC42DC52DBB0722080318220FCA2D11
:101B9200CB2DBC0723080318230ABD073D08AF005D
:101BA2003C08AE003B08AD003A08AC008A15482458
:101BB2008A15831203132809BE002909BF002A09C6
:101BC200C0002B09C100BE0A0319BF0A0319C00ACB
:101BD2000319C10A3E08B6073F0803183F0FF22D4A
:101BE200F32DB70740080318400FF82DF92DB80759
:101BF20041080318410AB9073908B5003808B4008A
:101C02003708B3003608B200062E08000A308312E5
:101C12000313A0000030A1002908A301A30728088C
:101C2200A201A2078A156C238A15831203132008C6
:101C3200013E84008A1500208A15AA002A08EA00BB
:101C42000A30A0000030A1002908A301A307280838
:101C5200A201A2078A11A5278A158312031321085C
:101C6200A901A9072008A801A8070A30A00000308E
:101C7200A1002908A301A3072808A201A2078A1527
:101C82006C238A15831203132008AA002A08AC00C9
:101C92000A30A0000030A1002908A301A3072808E8
:101CA200A201A2078A11A5278A158312031321080C
:101CB200A901A9072008A801A8070A30A00000303E
:101CC200A1002908A301A3072808A201A2078A15D7
:101CD2006C238A15831203132008AA002A08AB007A
:101CE200AB08031D752E762E972E1A3084008A15A6
:101CF20000208A15AA002A08E800AC08031D822EDB
:101D0200832E8C2E1A3084008A1500208A15AA0090
:101D12002A08E900AA2E2C08013E84008A15002018
:101D22008A15AA002A08E900AA2EAA2E2C08013E2A
:101D320084008A1500208A15AA002A08E9002B08C7
:101D4200013E84008A1500208A15AA002A08E800AC
:101D5200AA2E08000A3083120313D2005208A000F0
:101D62001330D3005308A10016308A1501228A15B8
:101D7200BB2EBB2E8A153F228A1500308312031315
:101D820021023D3003192002031CC82EC92EBB2E8E
:101D9200CA2E8A15BB218A158312031323088316C0
:101DA2000313AB0083120313220883160313AA0042
:101DB20083120313210883160313A900831203134A
:101DC200200883160313A80083120313EC15EA2ECE
:101DD200EA2E8A153F228A1500308312031321024C
:101DE2003C30031920020318F72EF82EEA2EF92EA2
:101DF2000030C9000030C8000030C7001E30C600E5
:101E02008A1529238A15F73083120313D200520848
:101E1200EC05ED01FC30D2005208EB05952F8A1536
:101E22003F228A1500308312031321023C3003192A
:101E32002002031C1D2F1E2F952F8A15BB218A15E8
:101E420083120313230883160313AF0083120313B1
:101E5200220883160313AE0083120313210883168C
:101E62000313AD0083120313200883160313AC007F
:101E7200280983120313D20083160313290983123C
:101E82000313D300D20A0319D30A831603132C08AF
:101E9200831203135207D400831603132D08031869
:101EA2002D0A831203135307D5006D08D600560777
:101EB200203E8400540883178000840A550880005D
:101EC200831603132F08AB002E08AA002D08A900C1
:101ED2002C08A80083120313EC15702F702F8A159B
:101EE2003F228A1500308312031321023C3003196A
:101EF200200203187D2F7E2F702F7F2F0030C90004
:101F02000030C8000030C7001E30C6008A152923E1
:101F12008A15F73083120313D2005208EC05013000
:101F2200D2005208ED07952F831603132809831256
:101F32000313D20083160313290983120313D30058
:101F4200831603132A0983120313D400831603137F
:101F52002B0983120313D500D20A0319D30A0319DA
:101F6200D40A0319D50A8A15BB218A1583120313D1
:101F72002008D20721080318210FC02FC12FD30731
:101F820022080318220FC62FC72FD40723080318CD
:101F9200230AD50700305502031DD92F0030540201
:101FA200031DD92F07305302031DD92FD0305202FF
:101FB2000318DC2FDD2FED2F24306D020318E22FE2
:101FC200E32FED2F6B18E62FE72FED2FEB1CEA2FF7
:101FD200EB2F102FED2FED2F6D08031DF12FF82F92
:101FE2006D08243A031DF62FF72FFC2FF82F01302E
:0E1FF200FF2FFF2FFF2F0030FF2FFF2F0800C3
:02400E00E4F0DC
:00000001FF
